:100000009FC00000B8C00000B6C00000B4C000002F
:10001000B2C00000B0C00000AEC00000ACC0000024
:10002000AAC00000A8C00000A6C00000B5C3000020
:100030005AC40000A0C000009EC000009CC0000088
:100040009AC0000098C0000096C0000094C0000054
:1000500092C0000090C000008EC0000007C20000E7
:100060008AC0000088C0000086C0000084C0000074
:1000700082C00000D704F904EB05F904EB053E0546
:100080005B05EB05AE05C0052E0341007200640060
:10009000750069006E006F00200044007500650067
:1000A0002000500072006F0067002E0020005000FA
:1000B0006F0072007400000032034100720064009F
:1000C000750069006E006F0020002800770077003F
:1000D00077002E00610072006400750069006E00F8
:1000E0006F002E0063006300290000000403090470
:1000F00009023E00020100C03209040000010202B0
:100100000100052400011004240206052406000154
:10011000070582030800FF09040100020A0000002D
:100120000705040240000107058302400001120197
:1001300010010200000841233D0001000102DC0122
:1001400011241FBECFEFD2E0DEBFCDBF11E0A0E093
:10015000B1E0EEE1F1E102C005900D92AA31B107E4
:10016000D9F722E0AAE1B1E001C01D92A833B2079D
:10017000E1F77BD0D2C744CFFC01E058FF4FA0810C
:10018000B1816C93A081B1819D012F5F3F4F31837D
:1001900020832E173F0721F412969C938E9311977C
:1001A0002FB7F894FC01EC57FF4F80818F5F80835D
:1001B0002FBF0895DC01AE57BF4FED91FC91119711
:1001C00021911196FC93EE93AC0140585F4FE417D8
:1001D000F50711F48D939C933FB7F894FC01EC570D
:1001E000FF4F9081915090833FBF822F08958823C5
:1001F00021F03F9A47985C9808953F9847985C9AF9
:100200000895882319F046985D980895469A5D9A56
:10021000089584B7877F84BF0FB6F894A89580911E
:100220006000886180936000109260000FBE80E0E3
:10023000DEDF469A3E9A87E690E09093CD00809369
:10024000CC0086E08093CA001092C80088E18093B9
:10025000C900539A5A9A8AB180638AB98BB1806374
:100260008BB98FD284E085BD0895D3DF2FB7F89482
:1002700087EA91E0909328028093270290932A02C4
:10028000809329022FBF2FB7F89482E291E09093D8
:10029000A3018093A2019093A5018093A4012FBF95
:1002A0007894D3E09FB7F89480912B029FBF803859
:1002B00049F084E091E0C2D697FD04C0682F87EA38
:1002C00091E05ADF8FB7F894C091A6018FBFA8992B
:1002D00003C0C13608F453C0A89A8091A6018823B0
:1002E00019F05D98D0931F01CC2349F082E291E090
:1002F00061DF682F84E091E042D6C150F5CF809154
:100300001F01882341F080911F01815080931F01BC
:10031000811101C05D9A80912001882341F0809174
:100320002001815080932001811101C05C9A80914D
:1003300002019091030118161906ECF4CC97853B45
:10034000910510F481E001C080E05BDF8091020143
:10035000909103010197C29710F481E001C080E001
:1003600046DF809102019091030101979093030170
:100370008093020104C080E044DF80E038DF9FB753
:10038000F89480912B029FBF882361F087EA91E067
:1003900011DF9091C80095FFFCCF8093CE005C9850
:1003A000D093200184E091E03BD608D57BCF84E058
:1003B00091E086C584E091E013C5CF92DF92EF9281
:1003C000FF92CF93FC018489813021F0823021F4A7
:1003D000C0E203C0C0E301C0C0E08389823009F4F9
:1003E000C8608589873031F0883031F0863029F453
:1003F000C26003C0C46001C0C6601092C900109200
:10040000C8001092CA00C784D088E188F28881E0D1
:1004100090EBC91694E0D906E104F10409F080E0FC
:1004200080931A01C701B60122E030E040E050E0BD
:1004300052D6CA01B90160587B47814E9F4FA70130
:10044000960127D6215031093093CD002093CC005E
:10045000C093CA0082E08093C80088E98093C900F5
:10046000CF91FF90EF90DF90CF9008951F920F9261
:100470000FB60F9211242F933F934F935F936F9377
:100480007F938F939F93AF93BF93EF93FF9360916D
:10049000CE008EB3843019F482E291E06DDEFF91DC
:1004A000EF91BF91AF919F918F917F916F915F91EC
:1004B0004F913F912F910F900FBE0F901F90189565
:1004C00020911E0120931D0130911C0130931B01CE
:1004D000FC018585982F917090931E0186958170FF
:1004E00080931C0180911A01882319F084EB90E01D
:1004F00006C0211108C0992331F082E390E0909367
:100500000301809302010895292F332722303105FA
:1005100059F02330310569F021303105E9F482E1E9
:1005200090E02EE231E01CC08EE390E020EF30E05E
:1005300017C099278130910549F028F0029761F49E
:10054000E8E8F0E005C0ECEEF0E002C0E8EBF0E037
:10055000849190E09F0104C080E090E020E030E0D2
:10056000FA01318320830895EF92FF920F931F9336
:10057000CF93DF93CDB7DEB72A970FB6F894DEBFDF
:100580000FBECDBF7E0126E0E20EF11CFE013196CA
:100590009F01870190E09093E9005091EC00D80111
:1005A0005D938D015091ED00D9015D939D019F5F99
:1005B000953089F7282F30E08701020F131FD801EB
:1005C0006C932E0F3F1FD9014C9391E09093E9005B
:1005D0001092F0001092E8001092ED002091EB00D4
:1005E0002E7F2093EB009F5F953081F790E0208174
:1005F00021FD0BC09F5F3196BFEFEB1AFB0A9530D0
:10060000B1F78093E90081E013C09093E900209155
:10061000EB0021602093EB00D7012C912093EC009C
:1006200020812093ED002091EE0027FDE3CF80E0B4
:100630002A960FB6F894DEBF0FBECDBFDF91CF91E3
:100640001F910F91FF90EF9008951092F40080E0B9
:100650008093E9001092F0001092E8001092ED00F3
:100660009091EB009E7F9093EB008F5F853081F738
:1006700008958091300287FF0FC08091E80082FDCD
:1006800004C08EB38111F9CF10C08091E8008B7740
:100690000AC08EB3882349F08091E80080FFF9CF2B
:1006A0008091E8008E778093E800089585E6909128
:1006B000EC0090FF05C09091E80090FF05C01BC0C2
:1006C0009091E80092FD17C09EB39923B1F09EB3BC
:1006D0009530A9F09091EB0095FD13C09091E10049
:1006E00092FFE5CF9091E1009B7F9093E1008150D4
:1006F000F1F684E0089580E0089582E0089583E0B3
:10070000089581E0089542D044D01EBA10922E027E
:1007100010922D0210922C0284E089BD89B582606E
:1007200089BD09B400FEFDCF8091D800982F9F7736
:100730009093D80080688093D800809163008E7F6A
:10074000809363008091D8008F7D8093D800809142
:10075000E0008E7F8093E0008091E1008E7F8093A7
:10076000E1008091E20081608093E2008091E100ED
:10077000877F8093E1008091E20088608093E200AF
:100780000895C1DF81E080932F0208951092E20066
:1007900008951092E10008951F920F920FB60F92E4
:1007A00011242F933F934F935F936F937F938F9376
:1007B0009F93AF93BF93EF93FF938091E10080FFEE
:1007C0001BC08091E20080FF17C08091E1008E7F06
:1007D0008093E1008091E2008E7F8093E20080911F
:1007E000E20080618093E2008091D8008062809373
:1007F000D80019BC1EBAFBD18091E10084FF29C04A
:100800008091E20084FF25C084E089BD89B58260C3
:1008100089BD09B400FEFDCF8091D8008F7D809303
:10082000D8008091E1008F7E8093E1008091E2000A
:100830008F7E8093E2008091E20081608093E200ED
:1008400080912E02811102C081E001C084E08EBB44
:10085000CED18091E10083FF27C08091E20083FF29
:1008600023C08091E100877F8093E10082E08EBB0E
:1008700010922E028091E1008E7F8093E1008091A2
:10088000E2008E7F8093E2008091E200806180939D
:10089000E200DBDE42E060E080E066DE8091F000B6
:1008A00088608093F000A3D18091E10082FF0AC0AC
:1008B0008091E20082FF06C08091E1008B7F8093EF
:1008C000E10095D1FF91EF91BF91AF919F918F91F1
:1008D0007F916F915F914F913F912F910F900FBE3C
:1008E0000F901F9018951F920F920FB60F92112420
:1008F000FF920F931F932F933F934F935F936F93A9
:100900007F938F939F93AF93BF93CF93DF93EF9397
:10091000FF93C9EED0E088818770F82E188200EF2F
:1009200010E0F8018081877F808378941DD0F8944F
:100930001882F801808188608083F882FF91EF91AE
:10094000DF91CF91BF91AF919F918F917F916F91E7
:100950005F914F913F912F911F910F91FF900F90B9
:100960000FBE0F901F9018951F93CF93DF93CDB7B5
:10097000DEB7AA970FB6F894DEBF0FBECDBFE0E397
:10098000F2E088E392E02091F10021938E179F0717
:10099000D1F78091300290913102492F50E04A30D6
:1009A000510508F018C1FA01E65CFF4FB0C380386A
:1009B00081F0823809F00FC18091340287708093F2
:1009C000E9008091EB0085FB882780F91092E9000F
:1009D00006C080912C0290912D029111826090911D
:1009E000E800977F9093E8008093F1001092F10067
:1009F000C0C0282F2D7F09F0EEC0882319F0823067
:100A000061F0DAC080913202813009F0D5C09330B4
:100A100009F080E080932D022BC080913202811179
:100A200027C080913402877009F4C6C08093E90022
:100A30002091EB0020FFC0C0933021F48091EB00A7
:100A4000806214C09091EB0090619093EB0021E0E4
:100A500030E0A90102C0440F551F8A95E2F7409388
:100A6000EA001092EA008091EB0088608093EB002E
:100A70001092E9008091E800877F7EC08111ABC0B1
:100A8000109132028091E800877F8093E800F1DDC9
:100A90008091E80080FD04C08EB38111F9CF8CC035
:100AA000812F8F7711F492E001C093E09EBB8068A4
:100AB0008093E30081C08058823008F08CC0809120
:100AC0003202909133028C3D53E0950779F583E033
:100AD0008A838AE289833FB7F894DE01139690E017
:100AE0002EE041E2E22FF0E040935700E49190FFC6
:100AF00003C0E295EF702F5FEF7080E38E0F8A33B3
:100B000010F0E95C01C0E82FF0E0ED93FD939F5FEA
:100B1000943141F73FBF8091E800877F8093E800E0
:100B20006AE270E0CE01019663D012C0AE014F5F61
:100B30005F4F60913402E8DCBC01892B09F43CC0B2
:100B40009091E800977F9093E80089819A81A6D0E0
:100B50008091E8008B778093E8002EC08038D9F52B
:100B60008091E800877F8093E80080912E02809337
:100B7000F1008091E8008E778093E8007ADD1CC058
:100B8000811129C0809132029091330299270297F6
:100B90009CF48091E800877F8093E8008091320286
:100BA00080932E0266DD80912E02811102C083E0C7
:100BB00001C084E08EBBFBDB8091E80083FF0DC0A9
:100BC0008091EB0080628093EB008091E800877F4A
:100BD0008093E80002C0EEDBEFCFAA960FB6F89440
:100BE000DEBF0FBECDBFDF91CF911F910895089555
:100BF00020913602309137022617370748F06115E9
:100C0000710539F42091E8002E772093E80001C0A7
:100C1000B90130E06115710561F12091E80023FD13
:100C200037C02091E80022FD2DC02EB3222391F180
:100C30002EB3253089F12091E80020FFEBCF2091E1
:100C4000F200FC01CF016115710549F0283038F43C
:100C500081918093F100615071092F5FF3CF31E0F2
:100C6000283009F030E02091E8002E772093E8004A
:100C7000D1CF3111D2CF06C08EB3882359F08EB3B5
:100C8000853051F08091E80082FFF6CF80E0089532
:100C900081E0089582E0089583E00895209136026E
:100CA000309137022617370748F06115710539F47E
:100CB0002091E8002E772093E80001C0B90130E0D0
:100CC0006115710569F12091E80023FD38C020917C
:100CD000E80022FD2EC02EB3222399F12EB3253039
:100CE00091F12091E80020FFEBCF2091F200FC0170
:100CF000CF016115710551F0283040F48491809343
:100D0000F100615071092F5F3196F2CF31E0283048
:100D100009F030E02091E8002E772093E800D0CF52
:100D20003111D1CF06C08EB3882359F08EB38530F0
:100D300051F08091E80082FFF6CF80E0089581E0D5
:100D4000089582E0089583E008956115710529F4FE
:100D50002091E8002B772093E8006115710511F1CF
:100D60002091E80023FD24C02EB3222319F12EB3D5
:100D7000253011F12091E80022FFEFCF2091F20001
:100D8000222331F301962091F100FC013197208359
:100D90006150710999F7DCCF8EB3882359F08EB377
:100DA000853051F08091E80080FFF6CF80E0089513
:100DB00081E0089582E0089583E00895CF938EB393
:100DC000882359F0C091E900C7701092E900809122
:100DD000E80083FDC9DDC093E900CF91089508952F
:100DE000CF93DF932091E80023FF67C0FC012081AF
:100DF00030E040913402509135024217530709F018
:100E00005CC0EC0180913102813251F018F48032E3
:100E1000E1F053C0823281F1833209F43EC04DC00B
:100E200080913002813A09F048C08091E800877FC4
:100E30008093E80067E070E0CF010F96D9DE8091E3
:100E4000E8008B778093E80038C0809130028132CF
:100E5000A1F58091E800877F8093E80067E070E06B
:100E6000CF010F9672DF8091E8008E778093E800C3
:100E7000CE01DF91CF91A1CA809130028132E9F495
:100E80008091E800877F8093E800F3DB8091320255
:100E90008D87CE01DF91CF9113CB809130028132CB
:100EA00061F48091E800877F8093E800E2DB609145
:100EB0003202CE01DF91CF9192CFDF91CF91089591
:100EC000CF93DF93EC01FC013D9689E0DF011D9299
:100ED0008A95E9F78C81811102C090E001C094E00D
:100EE0006A817B81898128E030E040E0261737075E
:100EF00020F44F5F220F331FF9CF4295407F92605D
:100F0000492B61E831DB8823B1F18885811102C06A
:100F100090E001C094E06E817F818D8128E030E017
:100F200040E02617370720F44F5F220F331FF9CF19
:100F30004295407F9260492B60E816DB8823D9F008
:100F40008C85811102C090E001C094E06A857B85A8
:100F5000898528E030E040E02617370720F44F5F0E
:100F6000220F331FF9CF4295407F9260492B61ECED
:100F7000DF91CF91F9CA80E0DF91CF9108950F936F
:100F80001F93CF932EB32430F1F4FC010785108911
:100F900021893289012B022B032BA9F0C62F8181D5
:100FA0008093E9008091E80085FF04C0C093F100C0
:100FB00080E00AC08091E8008E778093E80076DBBD
:100FC0008823A1F301C082E0CF911F910F91089572
:100FD0002EB3243019F5FC01478550896189728947
:100FE000452B462B472BD1F081818093E9008091DE
:100FF000F200882389F09091E8008091E8008E77D4
:101000008093E80095FD08C051DB811108C08091F4
:10101000E8008E778093E80080E0089582E00895EC
:101020002EB3243051F4FC014785508961897289BF
:10103000452B462B472B09F0CBCF08952EB32430F8
:1010400019F08FEF9FEF0895FC0147855089618962
:101050007289452B462B472BA1F385818093E900AC
:101060008091E80082FFEDCF8091F200882321F08B
:101070002091F10030E002C02FEF3FEF8091F200AD
:10108000811105C08091E8008B778093E800C90149
:101090000895A1E21A2EAA1BBB1BFD010DC0AA1FB9
:1010A000BB1FEE1FFF1FA217B307E407F50720F0D1
:1010B000A21BB30BE40BF50B661F771F881F991F4C
:1010C0001A9469F760957095809590959B01AC0195
:1010D000BD01CF010895052E97FB16F400940FD0A3
:1010E00057FD05D0D6DF07FC02D046F408C0509566
:1010F0004095309521953F4F4F4F5F4F0895909504
:101100008095709561957F4F8F4F9F4F0895EE0F9B
:0E111000FF1F0590F491E02D0994F894FFCF95
:10111E0014003200000340000004400000020800EA
:0A112E0000000000000000000000B7
:00000001FF
